:020000020000FC
:1000000018C935C20000000023C000004DC1000027
:10001000000050C1000000000000000002030406C0
:10002000080C101820304060800002030406080C01
:10003000101820304080FF000406080C10182030F3
:10004000406080A0C00005050D050D0602030302F7
:100050004FB662FD20C070FF1AC165FDFAC057FEA1
:1000600001C00994C0919700C395C0939700C5E063
:10007000C519B8F3D0919700CD1B98F3C8E7089441
:1000800083FDC795C4BDC52DCC2321F4C0E083FDFD
:10009000C0E8C4BD07C171FF03C09598AC98C09873
:1000A000C52D089483FDC795C4BDC09399006B7F8F
:1000B000C52DCF3F09F441C0C0919800C395C093AE
:1000C000980070FF35C09598AC98C0984FBE1895B1
:1000D0007860C091A000CC2391F0C0919800CA959F
:1000E000D091A000CD1B58F0777FC0919800D0919F
:1000F0009F00CD1B08F41CC02092980019C0959851
:10010000AC98C098C5E0CA95F1F7C0917500CA9542
:10011000C2FD09C0C1FD05C095FFAB9A95FD949A3B
:100120000EC0AD9A0CC095FF949A95FDAB9A07C08E
:100130009598AC98C0984FBE1895209299004FBEE4
:100140001895A5C0552021F095FF959A95FDC09A68
:10015000AC989DC0552009F0AC9A95FFC09895FDCC
:10016000959895C0552021F095FFC09A95FD959AD8
:1001700095FF959895FDC0988AC095FF949895FD38
:10018000AB9895FFAB9895FD9498C5E0CA95F1F7AB
:10019000552021F095FF959A95FDC09AAC9877C0AF
:1001A00095FF949895FDAB98AD98C5E0CA95F1F789
:1001B000552021F095FF959A95FDC09AAC9867C09F
:1001C000AD9895FF949895FDAB98C5E0CA95F1F769
:1001D000552009F0AC9A95FFC09895FD959857C0A9
:1001E000AD9895FFAB9895FD9498C5E0CA95F1F749
:1001F000552009F0AC9A95FFC09895FD959847C099
:1002000095FFAB9895FD9498AD98C5E0CA95F1F728
:10021000552021F095FFC09A95FD959A95FF9598E8
:1002200095FDC09834C095FFAB9895FD949895FFC7
:10023000949895FDAB98C5E0CA95F1F7552021F04B
:1002400095FFC09A95FD959A95FF959895FDC09854
:100250001EC082FF1CC0C0917500C2FD0BC0C1FD55
:1002600011C095FF949895FDAB9895FFAB9895FDBF
:1002700094980DC0C1FDF5CF95FF949895FDAB986E
:10028000AD9805C0AD9895FFAB9895FD9498C52D98
:10029000C095089483FDC795C4BDC0939900209272
:1002A000970064604FBE18954FB6C0E1C8BF6E7F1F
:1002B0004FBE18953FB68F7EABB7A074A211806178
:1002C000A0E0ABBFA9B7AE7FA9BF7894A0916600AC
:1002D000AA2349F0A92FAF7151F1A0916600AA9508
:1002E000A093660024C040E050E0A0B396FDA09526
:1002F000A2FD4FEF96FFA3E096FDA2E0A5BFAA27BF
:10030000A064AABF8D7FA0B396FDA095A2FD5FEF6C
:10031000451749F7A8E161FDA0936600A92FAF71C9
:1003200019F0A8E1A093660040938D008160A09130
:100330006700AA2331F0A0916700AA95A0936700F7
:1003400007C0A92FAF7121F08061AA27A064AABFBE
:1003500080FF48C0A0918D004A2F8E7FA92FAF71DA
:10036000C1F0403F08F040EFA42FA295AF704A0FB4
:100370005091B000533069F0A695A69550FD01C08C
:10038000A69552FD03C0A41B4A2F03C04A0F08F4D0
:100390004FEFA09196004A1708F44A2F409361004E
:1003A00071FF08C0A091610050919200A51710F054
:1003B00050936100A091610040916300A41B70F014
:1003C0004091CF00A40B50F0A0916300A40FA09324
:1003D000630040F4AFEFA093630004C0A0916100FC
:1003E000A093630040916300A09192004A1708F027
:1003F0004A2F542EA52DA03408F06860A09160000B
:10040000A395A093600051F0F894A9B7A160A9BF8B
:1004100084FF02C0A0E4ABBF3FBE189541E05091FD
:100420006600552331F0A92FAF7119F45A955093F6
:100430006600A0918D00A13018F0209290000DC0B0
:100440002092910020929A00A0919000AF5FA0931B
:10045000900018F0AFEFA0939000F894A9B7A160B6
:10046000A9BF84FF02C0A0E4ABBF3FBE18953FB652
:100470004CB55DB58F7EABB7A074A2118061A0E0D2
:10048000ABBFA9B7AE7FA9BF789481FD26C096FF08
:10049000A2E096FDA3E0A5BF8260A0B396FDA09563
:1004A000A2FF05C0409364005093650033C196FFDE
:1004B000A3E096FDA2E0A5BFAA27A064AABF8D7FF6
:1004C000A92FAF7109F417C140E0A0B396FDA09524
:1004D000A2FD11C140938D0004C196FFA3E096FDDB
:1004E000A2E0A5BF8D7F61FF6BC096FFA2E096FDE5
:1004F000A3E0A5BFAA27A064AABF8260409388009A
:1005000050938900A09086004A19B09087005B093B
:10051000BB24A2E0EA2EA22C483CA0E05A0730F40B
:10052000A0E1BA2EE22CAAE0AA2E27C04836A1E00C
:100530005A0730F4A8E0BA2EE22CAFE0AA2E1DC074
:10054000403DA2E05A0730F4A4E0BA2EE22CAEE11E
:10055000AA2E13C0403AA5E05A0730F4A2E0BA2E02
:10056000E22CACE3AA2E09C04839A8E05A0728F4C7
:10057000A1E0BA2EE22CA8E7AA2EC42EA0918A00F0
:10058000CA1AD52EA0918B00DA0ADD202AF4AFEF2B
:10059000C094D094CA1ADA0A20928C00CA14DE04DD
:1005A00018F4A1E0A0938C0040938A0050938B0034
:1005B00040918800509189004093860050938700B5
:1005C000A09164004A1BA09165005A0B94FD7CC069
:1005D00093FD7AC092FD76C05695479591FD72C005
:1005E0005695479590FD6EC0D52EC42ED694C794CF
:1005F00061FD0CC0AC2DAC51AD2DA24008F07BC00C
:10060000DD2021F4AC2DA85C08F475C0A0E0EA2E32
:1006100097FD08C0E090C200A091B400A33011F48F
:10062000E090CA00AAEFEA0EF22CF21CCE18DF0806
:100630004FB74170A091B400A330A9F4442329F02E
:1006400095FD11C0F894906204C095FF0CC0F89419
:100650009F7D9598AC98C0989498AD98AB9871FD93
:1006600001C060687894442369F0A091B400A3307D
:1006700031F4AFEFC094D094CA1ADA0A03C040E054
:1006800050E022C0A091B400A33049F4CC0CDD1C92
:10069000A5E0CA1AD20818F4A0E0CA2ED22CAFEFF7
:1006A000CA16D20418F04FEF50E00EC0F090A70029
:1006B000CF9C412D000C441F50E008F012C04FEFBA
:1006C00050E00FC05695479594FF07C0552309F099
:1006D0004FEFA42FA6954A0F521D4F3F520508F029
:1006E0004FEF40938D00816061FF05C0AFE1A095A1
:1006F000A923AB299A2FA8E1A0936600A92FAF7177
:1007000019F4AAE0A093660061FD04C0A92FAF719F
:1007100009F08F7EA6E0A0936700A92FAF7119F4AE
:10072000AAE0A0936700F894A9B7A160A9BF84FFCD
:1007300002C0A0E4ABBF3FBE189511E00AC013E0B1
:1007400008C01AE006C01EE104C014E602C018EC9E
:1007500000C005E1BB27BA95F1F70A95D9F71A95BC
:10076000C1F708952AE338E709C020E33CE806C052
:100770002AE234EB03C025E238EC00C0652CB1E07E
:100780005B2E12E095FD9F7D95FF9062BB27AD9893
:10079000BA95F1F7552009F0AC9ABA95F1F7AC98F3
:1007A000BA95F1F7AD9ABA95F1F7552021F095FF7A
:1007B000959A95FDC09AB091A800BA95F1F795FF6A
:1007C000959895FDC098B7E8BA95F1F71A95D1F6C6
:1007D000022FB22FBA95F1F70A95D9F73A9571F62B
:1007E000AD98562C0895221B39E0001F3A9509F464
:1007F0000895221F211B18F4210F8894F6CF089426
:10080000F4CF622C722CB0E08894B395221F331F72
:10081000E0F7379527958894912E802E020B130BC5
:1008200010F4192D082D10F4889401C00894661C4A
:10083000771CBA9571F7172D062D0895322D1123C7
:100840002AF43A9500951095031B130BF894029F18
:10085000712C002D129F912C802C7894780C172DE0
:10086000921C292DB4E06B2E2695179507956A9456
:10087000D9F7332321F000951095031B130B08952E
:10088000089566FF21C010917400169500917300C1
:100890000795B0917700B01B0B2FB0917800B10B8A
:1008A0001B2F28F40038BFEF1B0740F009C00F379B
:1008B000120508F405C00FE710E002C000E81FEFC2
:1008C00000937C0010937D00089566FF39C000916D
:1008D0007C00B09179000B0F10917D00B0917A00EF
:1008E0001B1F20E030917D0033230AF42A95B0913C
:1008F0007B002B1F1AF4203F40F00AC02F3008F471
:1009000007C00FEF1FEF2FE003C000E010E020EF63
:1009100030916300B09192003B1718F4332331F00B
:1009200009C0B0917D00BB235AF004C0B0917D0096
:10093000BB2332F40093790010937A0020937B005C
:10094000089566FF2FC02091CD0000917C00000F1C
:1009500010917D00111F72DF11232AF40038BFEFC0
:100960001B0740F009C00F37120508F405C00FE758
:1009700010E002C000E81FEF002352F0B0916200C7
:10098000B01B0B2F18F0013008F00AC001E008C0BE
:1009900000950F5FB09162000B0F08F001C00FEFE0
:1009A00000937E00089566FF2DC02091CE00009137
:1009B0007A0010917B0042DF11232AF40130BFEF4F
:1009C0001B0740F009C00F3F120508F405C00FEFE8
:1009D00010E002C001E01FEF112352F0B0917E0041
:1009E000B01B0B2F18F0013008F00AC000E008C05F
:1009F00000950F5FB0917E000B0F08F001C00FEF64
:100A00000093630008950FEF677FB72FB670E9F486
:100A10006860B0917400B83008F0677FB0917400DE
:100A2000A1F00FEF10917400DEDEF894B091700029
:100A30000B9F112D002D7894112309F00FEFB09129
:100A400095000B1710F40091950000939400089501
:100A50006BC0D9D274FFB2E074FDB1E0B7B9B6B1E2
:100A6000B068B064B6B969DE74FFB2E074FDB1E09D
:100A7000B7B9B6B1B068B064B6B9B6B1B6FDFDCF1E
:100A800004B115B1B6B1BF77B6B902D324E720934C
:100A9000A30030E03093A400732E7694622E669407
:100AA000620E731E262D372D0217130778F08090E3
:100AB000A300B4E7B80DB093A3008090A400B0E009
:100AC000B81DB093A400260D371DEECF8090A30073
:100AD0009090A4001091A40016950091A300079592
:100AE00016950795B091A300B00FB093A100B091F7
:100AF000A400B11FB093A20023E0169507952A9594
:100B0000E1F72091AF002A9529F42092A3002092CA
:100B1000A4000AC02A9521F0800E911E2A95E1F7C3
:100B20008092A3009092A40008952091AF00B6B1E6
:100B3000B6FDFBCF04B115B1B6B1BF77B6B9B09170
:100B4000A500B395B093A500B83060F12092A50040
:100B5000B091CC00BB2321F1112329F0B091A60064
:100B6000BF3F61F009C0B091A6000B1739F020F427
:100B7000BB2321F0BA9502C0B395E1F30091920036
:100B8000B093A600B83850F400ECBD3738F400E854
:100B9000B23720F400E4B73608F400E00093920086
:100BA0007F7E0895B0919200B39511F0B0939200BA
:100BB000B091A500B73009F47061089502E3F8948C
:100BC000B091D0000B9F012D000C001F7894B091C4
:100BD00092000B1710F000919200009361000093B7
:100BE0006300502E00939500089520927300B8E0A2
:100BF000B093740008952091800030918100F894A2
:100C00000CB51DB5200F311F3BBD2ABD6160B0E1A1
:100C1000B8BF7894209171003091720000937100F8
:100C200010937200021B130B20917300309174001B
:100C3000622E732EB4E08B2EB2E09B2EB091740026
:100C4000B43010F08A949A94B83010F08A949A9440
:100C5000769467948A94E1F726193709992021F050
:100C6000169507959A94E1F7200F311F2093730092
:100C70003093740008F00895BFEFB0937300B09301
:100C8000740008952091820030918300F8940CB58F
:100C90001DB5020F131F1BBD0ABD6160B0E1B8BFD7
:100CA0007894089560FDFECFEDDF0895B091BE0009
:100CB00000916E00023808F0B395003A08F0B39541
:100CC000B63008F0B5E09B2EBCE08B2EB0917400DE
:100CD000B33030F48394839482FF02C0839483946E
:100CE000B23030F48394839482FF02C0839483945F
:100CF00071FF03C0B3E09B2E822C10917400009111
:100D0000730024E0169507952A95E1F70819120952
:100D100028F0B02FB250B12FB20910F402E010E069
:100D2000312F202F712E602E76946794B92DB33019
:100D3000E9F0B0FD05C0060D171D262D372D06C0A4
:100D4000000F111F0250120922E030E0B92DB3301C
:100D500068F0209384003093850000938000109306
:100D60008100609282007092830008950093840055
:100D70001093850020938000309381006092820060
:100D800070928300089560FDFECF20918200220FB3
:100D900030918300331FB72FB67021F0209173007C
:100DA00030917400F8940CB51DB5020F131F1BBDD4
:100DB0000ABD6160B0E1B8BF789408956061209287
:100DC000760020E004C060612092760020E2B72F18
:100DD000B67009F06F7E789460FD05C0B091760022
:100DE000BB2309F0089501E063FF0AC0B0917400CD
:100DF000B33008F002E0B0917400B63008F003E0C0
:100E000071FF01C006E060FD06C0B0917600BB2313
:100E100011F0789408951AE083FF1AE078940000A6
:100E20000000F89462FD03C014E183FF14E171FF38
:100E300001C018E7B4B530919900B31BB10B18F39A
:100E4000B0917600B395B0937600B5E03B2F6B2E52
:100E5000722CB8B1B072B21709F073943A95C9F711
:100E60007394761488F464FFB2CF6F7E3CB56DB492
:100E70007090730080907400370D681C6BBC3ABD95
:100E80006160B0E1B8BFA3CF64FDA1CF0A9509F0BE
:100E9000BACF7894089571FF0AC0B0916D00B395F0
:100EA000B0936D0060FD0CC020926D0009C060FD24
:100EB00007C064FD05C067FD03C0BF91BF914EC46C
:100EC00008952091840030918500F8940CB51DB5EB
:100ED000020F131F1BBD0ABD6160B0E1B8BF78945B
:100EE0000895EFDF00E063FF03C064FF01C001E08D
:100EF000F89410916E00B7E01B9F212D102D78946F
:100F0000200F2695179526951795269517951093DA
:100F10006E00183718F4B8E7B0936E0000916E00B9
:100F2000B0916F000B1720F060629598AC98C09854
:100F300060FDFECF0895F8949498AD98AB9882FF29
:100F400007C0E0E0F1E073FF03C0BEE1BA95F1F73E
:100F500095FF949A95FDAB9AB2E0B093750089C065
:100F6000F89495FFC09895FD959882FF0DC0E0EF2D
:100F7000F0E073FF0BC0AD9895FFAB9895FD94988A
:100F8000BEE1BA95F1F702C0EAEAF0E062FF03C001
:100F9000552009F0AC9AB3E0B09375006AC0F8949C
:100FA0009498AD98AB9882FF07C0E0EEF0E073FF35
:100FB00003C0BEE1BA95F1F795FFAB9A95FD949AFF
:100FC000B4E0B093750055C0F894AC9882FF0DC0A2
:100FD000E0EDF0E073FF0BC095FF949895FDAB98A2
:100FE000AD98BEE1BA95F1F702C0E2EAF0E062FF27
:100FF00006C0552021F095FF959A95FDC09AB5E061
:10100000B093750036C0F8949498AD98AB9882FF71
:1010100007C0EDEBF0E073FF03C0BEE1BA95F1F756
:10102000AD9AB6E0B093750024C0F89495FF9598FA
:1010300095FDC09882FF10C0E3E1F1E073FF0EC0A0
:1010400095FF949895FDAB9895FFAB9895FD949876
:10105000BEE1BA95F1F702C0E2EBF0E062FF06C034
:10106000552021F095FFC09A95FD959AB1E0B09377
:10107000750067FF0AC00CD0BEE1BA95F1F7B5E084
:10108000BA95F1F7949AAD9AAB9A6F7D78940895DA
:1010900021EA30E0F9019598AC98C0989498AD9801
:1010A000AB986B7F0895ACEAB0E00FEF0D930D9312
:1010B0000D930D9303E00D9304E00D930BE00D935E
:1010C00001E00D9301E00D9301E00D93A8EBB0E07A
:1010D00001E00D930FEF0D930D930FEF0D930D9313
:1010E0000D9303E00D9306E00D930FEF0D930D9319
:1010F00005E20D9300ED0D930AEF0D930AEF0D93AA
:1011000004E00D930DE00D9301E00D9300E00D93CD
:101110000AE70D930FEF0D9301E00D9308952091D1
:10112000BF0009E011E0223011F405E011E02330A6
:1011300011F405E012E0243011F405E013E025304D
:1011400011F409E017E0263011F400E010E00093FC
:101150009F001093A0002091B3008B7F777FB09108
:10116000B400B33019F09F7DB1FD90629F7BB091C8
:10117000B500B1FD9064B22FB23011F0886001C0AB
:10118000877F0895ECE1F0E00091AC000A95E00F54
:10119000F21DB491B093CD000091AD000A95E00F1F
:1011A000F21DB491B093CE0073DF0895EAE2F0E04F
:1011B0000091C7000A95E00FF21DB491B093CF00E3
:1011C00067DF0895E8E3F0E00091B2000A95E00FD0
:1011D000F21DB491B093D0005BDF08950895B091F3
:1011E000C8000FEF1CE0B23011F400EA1AE0B3308F
:1011F00011F402E815E000936F0010937000089559
:1012000008952091C2003091C30097FF02C020E0F2
:101210003FEFB32FB21B6B2EB25810F4B2E86B2E17
:1012200000E00395609EB12DB058D8F30093A7005D
:101230000895F894E3E0F0E0B9E0B7BFB491B07876
:10124000C1F3F894A895B1B5B861B1BDB0E0B1BD36
:10125000B4E0BEBFBFE5BDBF1BDFB0E0B8BBB1E1CE
:10126000B7BBB0E0B5BBB8E3B4BBB0E0B2BBB0E372
:10127000B1BB2224A0E0B0E02D92AA31E9F7A0E6AC
:10128000B0E00FEF2D920A95E9F70DDF87D247DF27
:1012900079DF8CDF97DFA2DFA2DFB2DFB2DF009160
:1012A000C4000093A800F4DEB2E0B3BFB2E0BEBD5C
:1012B000B2E0B5BDF8944BDA55DA45DA56DA43DADE
:1012C00057DA41DAF6D243DA42DA3FDAB1E5B8BFAB
:1012D000B9BFB0B7B860B0BFB6B1B460B6B92DDAB7
:1012E0007894B6DBB0E4BBBFBB27B064BABF8D7FD8
:1012F0002EDAB1E0B0936900626025E0B0918C0015
:10130000BB2309F425E01BDAB0918D00B230A8F3BD
:10131000B92FBF7100918F0000938E00B0938F00A2
:10132000B01759F72A9551F76D7F96FFB3E096FDF8
:10133000B2E0B5BFBB27B064BABF8D7F06DAFFD974
:1013400002E0B92FBF7109F400E0B0918D00B01731
:10135000B0F3F89407DA06DA05DA7894F8D920922F
:101360007F00B091B400B33009F472C0E8D9B091F5
:10137000B800B13008F46CC0B0916900B13008F425
:1013800067C0B92FBF71C1F0B0918D00BF3F08F4A5
:101390005FC0F894F0D97894D8D9B0918D00B1306D
:1013A000C0F7F894DFD9CDD9DDD97894CED9B091F2
:1013B0008D00BF3FB0F3AFC2B8E09B2E9068F894A9
:1013C00020DF7894C2D9F8949F771BDF80908D003E
:1013D000B0918D00BF37789408F442C0AED9F8942C
:1013E000CAD978949A9451F7B82DB550B093C300E8
:1013F000AED9F89400D262D27894BAE09B2E90686D
:10140000F894FFDE7894A1D9F8949F77FADE809063
:101410008D00B0918D00BF37789478F78ED9F8940D
:10142000A1D98FD99FD978949A9449F7B82DBB5FE9
:10143000B093C2008CD9F894DED14FD2789485D97C
:10144000F894DFDE7894B0918D00BF3FC0F363C2A3
:1014500000918D00B0917F000B1710F000937F007A
:1014600074D901E0B091B400B35009F405E0B09133
:101470008D00B01708F075CFF8947DD97CD97BD951
:10148000789465D92092690020926A0020926B00BE
:10149000B0916A00B395B0936A00BF3F69F5B0910F
:1014A0006B00B395B0936B00B091C60009E1BA959B
:1014B00059F002E3BA9541F00DE7BA9529F00AEF29
:1014C000BA9511F020926B00B0916B00B017A0F0AC
:1014D000B0916B00BA95B0936B00B4EBB0936A0017
:1014E000B091C500B093A800F89445D97894B09114
:1014F000C400B093A80029D924D9B0916600BB23B9
:1015000021F4B92FBF7109F4F7CEB0918D00B63038
:1015100008F4BECFB091B400B35009F016D9B09121
:101520006600BB2309F4E8CEF894B2DD2092610096
:101530002092620020926300522C7894B091B10006
:10154000B093960020927700209278002092790044
:1015500020927A0020927B002092A50060E070E04B
:1015600020926E0042DBB8E0B093A5007061E5D830
:1015700074FFB2E074FDB1E0B7B9B6B1B068B06461
:10158000B6B9B6B1B6FDFDCF04B115B1B6B1BF77EE
:10159000B6B9112309F00FEF0093A600C6DAB8E040
:1015A000B093A50070618090B300B2E0B093B30037
:1015B000B6DD8092B300F894BFEFB0939200FEDAEC
:1015C000B0916100B0939200B0939300B0939400F7
:1015D0007894B1E0B0936100B09363005B2EB09358
:1015E0009B00B0919100B0939A007160726020925C
:1015F0006D0009DD1ADDFFDAF8DA58DB04C08FDD93
:101600002092A5007F7E95FFB6E095FDB0E0B7B9CA
:10161000DADB41DC56DC34D964DC8DDCECDA42DB2D
:1016200045DBB1DBB7E0B7B9C9DB35DC4ADC29D92A
:10163000EAD957DC95DCDFDA35DB38DBA4DB95FF54
:10164000B0E095FDB6E0B7B9BEDB25DC3ADC3DD9AC
:1016500048DCA5DCD0DA26DB29DB95DB95FFB6E09C
:1016600095FDB0E0B7B9AADB16DC2BDC6AD939DC12
:10167000ABDCC1DA17DB1ADB86DBB7E0B7B9A3DB7B
:101680000ADC1FDC90D92DDCBEDCB5DA0BDB0EDB0F
:101690007ADB95FFB0E095FDB6E0B7B98FDB74FF5C
:1016A000B2E074FDB1E0B7B9B6B1B068B064B6B934
:1016B000F2DB07DC16DCB9DC9EDAF4DAF7DA35DACD
:1016C00062DB71FF25C067FD23C0B0919500B09328
:1016D0009200B0939300B0919100B0939A00B1E062
:1016E000B0939B0014E624E1B0916D00B11750F067
:1016F0007D7F746020936C00BFEFB0939200B09335
:10170000930006C0B0918D00B13008F07CCF26C0A8
:1017100072FF10C067FD0EC0B0916C00BA9511F455
:101720007B7F6DCFB0936C00B0918D00B13008F02D
:101730006ACF14C0B0919000B23880F4B92FBF7155
:1017400021F4B0916600BB2349F0B091740000EF22
:1017500067FF01C000E6B01708F455CFF89498DC95
:101760008090B300B2E0B093B300D9DC8092B300B4
:10177000209261002092620020926300522C2092FD
:1017800096007E7F7894D9D783DCB92FBF7129F476
:10179000B0916600BB2309F4AFCD76CEEDE0F0E06A
:1017A00023D00A3509F01BC0EEE0F0E01DD0053A69
:1017B00009F015C03AE0ACEAB0E0E3E0F0E014D0A4
:1017C0000D9331963A95D9F735E1A8EBB0E0EFE00B
:1017D000F0E00AD00D9331963A95D9F702C063DC58
:1017E0000AD0E4E2F0E00895E199FECFEEBBFFBB42
:1017F000E09A0DB308951ED03AE0ACEAB0E0E3E021
:10180000F0E00D910FD031963A95D9F735E1A8EB7C
:10181000B0E0EFE0F0E00D9105D031963A95D9F7C0
:1018200012D00895E199FECF0DBBEEBBFFBBE29A4B
:10183000E19A0895EDE0F0E00FEFF4DFEEE0F0E084
:101840000FEFF0DF0895EDE0F0E00AE5EBDFEEE00A
:10185000F0E005EAE7DF08953091A9000091AA00C1
:10186000313011F40093B000323011F40093B10024
:10187000333011F40093B200343011F40093BE0001
:10188000353011F40093C700363011F40093BF00D7
:10189000373011F40093B300383011F40093C800CE
:1018A000393011F40093B4003A3011F40093B500CC
:1018B000089525E04CD72A95E9F7089553D755D7D1
:1018C00057D759D73ED74ED750D752D754D739D7F5
:1018D00049D74BD74DD74FD708954DD749D745D77F
:1018E00041D72FD748D744D740D73CD72AD743D75B
:1018F0003FD73BD737D708958090A9009090AA0092
:1019000031D730D72FD71DD78A94D1F734D719D7ED
:101910009A94E1F70895F894D1DF7894CADFC9DF8B
:10192000B1E0B093A900B1E0B093AA002092AB005F
:10193000F894E2DF7894B5E06B2E70908D0007D7B5
:10194000B0918D007B16C9F7B13018F0BF3F40F160
:1019500007C082DFF8944FDFB1DFB8E0B1BDA9DF87
:101960006A9459F7B091AB00B395B093AB00B33024
:1019700008F4DECF9EDFB091AA00B395B093AA0021
:10198000F894B091A900BA95E6E4F0E0EB0FF21DEF
:10199000049178940395B091AA00B01708F4C6CFCB
:1019A00088DF87DFB091A900B395B093A900B0910B
:1019B000A900BB3008F4B7CF76DBF8941CDFB8E0A1
:0419C000B1BD77DF5F
:00000001FF
